:020000040000FA
:1000000000000B1A5C2809288B184F200B192C2094
:1000100009000130A7008500073099008316FC30E5
:1000200085000113811381118112011081100111CA
:100030000B16FF2390000B123430950083124F20D3
:100040000301851A40308316810483128B100B1133
:100050000B168B168B172B280B11051E0800FF3073
:10006000A107031CA207031808002030A007A13035
:100070000318A130A1070730A200A50B0800A603B2
:10008000260F08006520A5006520A6002506031D93
:100090004B28602042282709A70085000800FE3071
:1000A000A700270985008B1060202030A000A13018
:1000B000A1000730A20042288312033085005F2888
:1000C0000030A4006C30A300080024088A00230834
:1000D000A30A0319A40A8200013400340234003454
:0C00E000013400340334003400340034D8
:02400E00A43FCD
:00000001FF
